:10000000D00C002019130000F13900004913000042
:100010004913000049130000491300004913000070
:100020000000000000000000000000005D11000062
:10003000491300000000000005110000C93900004C
:10004000D9120000D9120000D9120000D912000004
:10005000D9120000D9120000D9120000D9120000F4
:10006000D9120000D9120000D9120000D9120000E4
:10007000D9120000D9120000D9120000D9120000D4
:10008000D9120000D9120000D9120000D9120000C4
:10009000D9120000D9120000D9120000D9120000B4
:1000A000D9120000D9120000D9120000D9120000A4
:1000B000D9120000D9120000D9120000D912000094
:1000C000D9120000D9120000D9120000D912000084
:1000D000D9120000D9120000D9120000D912000074
:1000E000D9120000D9120000D9120000D912000064
:1000F000D9120000D9120000D9120000D912000054
:10010000D9120000D9120000D9120000D912000043
:10011000D9120000D9120000D9120000D912000033
:10012000D9120000D9120000D9120000D912000023
:10013000D9120000D9120000D9120000D912000013
:10014000D9120000D9120000D9120000D912000003
:04015000D9120000C0
:1001540053B94AB9002908BF00281CBF4FF0FF312A
:100164004FF0FF3000F070B9ADF1080C6DE904CE2A
:1001740000F006F8DDF804E0DDE9022304B070477E
:100184002DE9F047089E0D4604468A46002B7FD190
:100194008A42174641D9B2FA82F24AB1C2F1200129
:1001A40005FA02F39740944020FA01F141EA030A68
:1001B4004FEA17484FEA144C1FFA87F9BAFBF8FEC6
:1001C40008FB1EA30EFB09F14CEA0343994206D92E
:1001D400FB1802D2994200F224810EF1FF3E591A13
:1001E400A3B2B1FBF8F008FB101100FB09F943EAD4
:1001F4000144A14505D93C1902D2A14500F20E8162
:100204000138A4EB090440EA0E4000211EB1D44099
:100214000023C6E90043BDE8F08702B9FFDEB2FA65
:1002240082F2002A4FD1CB1B4FEA174E1FFA87F8F0
:100234000121250CB3FBFEFC0EFB1C302B4608FBF6
:100244000CF945EA0045A9450AD97D192CBF0123BB
:100254000023A94502D9002B00F0D9800CF1FF3C02
:10026400A5EB0905A3B2B5FBFEF00EFB105508FB88
:1002740000F843EA0544A04505D93C1902D2A0453B
:1002840000F2C9800138A4EB080440EA0C40BDE741
:100294008B4208D9002E00F0B1800021C6E9000588
:1002A4000846BDE8F087B3FA83F1002946D1AB4292
:1002B400C0F0A780824240F2A4800846002EAAD053
:1002C400C6E9004AA7E7C2F12000974001FA02F309
:1002D4004FEA174EC14024FA00F51FFA87F89440FC
:1002E4001D43B1FBFEF02B0C0EFB101100FB08FCB0
:1002F40043EA01439C4509D9FB182CBF0121002185
:100304009C4502D9002900F095800138A3EB0C0329
:10031400ADB2B3FBFEF10EFB113301FB08FC45EA61
:100324000345AC4505D97D1902D2AC4500F289805C
:100334000139A5EB0C0341EA00417AE7C1F120043D
:100344008B4002FA01F705FA01FCE24020FA04F8B6
:10035400E54000FA01FE134348EA0C024FEA134851
:100364004FEA124C1FFA83F9B5FBF8FA08FB1A5549
:100374000AFB09F04CEA054C60450AD913EB0C0C56
:100384002CBF01250025604501D9002D55D00AF167
:10039400FF3AACEB000C92B2BCFBF8F008FB10CCBB
:1003A40000FB09F942EA0C4CE14505D913EB0C0CAE
:1003B40001D2E1453BD8013840EA0A40ACEB090CD4
:1003C400A0FB0789CC4545464A4602D306D1C6451B
:1003D40004D20138B8EB070569EB03022EB3BEEB78
:1003E40005036CEB020C23FA01F20CFA04F42CFA68
:1003F40001F300211443C6E900430CE731463046BB
:1004040009E7841A65EB030301209A4656E7ACF129
:10041400020C3D4424E702383C4434E702383C44AF
:10042400EFE6AEF1020E3B44D9E63146F3E602387C
:100434009C44C1E702383B4468E7AAF1020A9C44A1
:10044400A7E702393D4474E7704700BF70B5174809
:1004540001F01EFF044620B3C568836840F20162C0
:100464001C211B68984700281AD12B6843F080533D
:100474002B600125E36885F001061B6813F0805F9B
:1004840018BFF5B275B1A368DB684FF08051204600
:100494009847F5B200214FF4004002F07BFCE9E7F5
:1004A400E7DA70BDA3681B69EFE700BF20440000D2
:1004B4002DE9F04F87B00F461946109B06461425C8
:1004C400104698469DF844B09DF848A01E4C4FEA4B
:1004D400E37950EA01031AD1142D08BF3023139C89
:1004E40018BF01352C4408BF8DF81430152C1BD0CF
:1004F400153C002C1ADC1DF8050039460135B047BF
:10050400152DF8D1002C19DC07B0BDE8F08F424658
:100514004B46FFF71DFE84460B46A25C60460DF871
:1005240005201946013DD4E70024E4E7BBF1000FA0
:10053400E1D039465046B047013CDAE739465046E7
:10054400B047013CDEE700BF274400000B680133DD
:100554000B60014B1B68184700000020014B18601A
:10056400704700BF000000202DE9F04F002605462B
:100574008B461C464FF0FF38374687B002F1FF3AEE
:100584004FF0000907E0B9F1000F0BD1252800F066
:100594000A815946A8471AF8010F0028F3D107B079
:1005A400BDE8F08F7A280AD8622810D8302851D0B4
:1005B40044D8252800F0F5802D2800F0FB8059460A
:1005C4002520A84759469AF80000A847D8E7A0F183
:1005D4006303172BF3D801A252F823F09F070000FE
:1005E400A1060000C3050000C3050000C305000008
:1005F40083060000A1060000C3050000C305000037
:1006040083060000C3050000C3050000C305000005
:100614001B070000C3050000C305000067070000B6
:10062400C3050000A1060000C3050000C3050000C7
:1006340049060000C305000083060000392815D9C7
:100644005828BCD19AF80030702B6ED1002354F88E
:10065400042B75E0B8F1000F0BDA002F00F0AC802A
:10066400A0F13008002F08BF022794E7B8F1000F6B
:10067400F6DB0A2303FB0808A8F13008F2E7682830
:1006840003D1682E06D1482685E76C2802D16C2E4A
:1006940000F09480002E92D106467CE77A2E06D193
:1006A400A14659F8042BD317752823D10FE06C2EDB
:1006B400F6D04C2E05D1073424F00709F9E80223BB
:1006C400F2E77528226804F1040912D10023F81E08
:1006D40018BF0120012F0CBF3024202401900A20D0
:1006E400CDE90248009059462846FFF7E1FE4C4602
:1006F40046E7D317002A73F10001E8DA59462D20A2
:10070400CDE90423A847DDE90423524263EB430304
:1007140008F1FF38DBE759463020A84759467820CE
:10072400A8474FF0080801278CE76C2E8ED04C2E7A
:100734008CD1E31D23F007031C465B6854F8082B97
:10074400F81E18BF0120012F0CBF30212021CDE954
:10075400021810210190009128465946FFF7A8FE7F
:100764000EE754F8043B99464A4619F8010B78B948
:10077400032F25D1A2EB0309A8EB0909B9F1000F56
:100784007FF7FEAE59462020A84709F1FF39F5E767
:1007940059460493A847049BE6E7594654F8040BCA
:1007A40013E7594611E74E464F464FF0FF384FF0D6
:1007B4000109F0E60327EEE60127ECE64C26EAE61B
:1007C4008146E8E607B50B4600210246019103483D
:1007D40001A9FFF7C9FE03B05DF804FB5105000051
:1007E4002DE9F84FB0F81890044619F0080893461C
:1007F4000DD001290CBF49F0100949F02009A0F8D7
:1008040018908BF31188BFF36F8FBDE8F88F09F050
:100814000709022907D1204602F085FE0028F0D0FE
:100824000128238B50D16769218B002F15DA2568A5
:1008340021F00701C4E9008841F001012183002669
:10084400218B01F0070ACA4502D0A368002B5CD1B2
:100854000DB9002E74D0002358E001F007035A1F8D
:10086400012A20D821F00701062B256889B2C4E9A2
:1008740000880CD1002D2B4638BF00232BB1628B8E
:100884001B6801326283002BF8D141F0020120463B
:10089400218302F048FE06460028D1D0238B43F082
:1008A40020032383CBE7042B0CD121F0070189B269
:1008B4002046218302F037FE05460028BFD041F0D0
:1008C400200121830025BAE7032809D1226923F0F6
:1008D4000703166843F00603002523832F46AFE77A
:1008E400042806D1226923F00703566843F0040361
:1008F400F2E7052806D1226923F00703966843F03E
:100904000503E9E700252E46E8E7012341F0080145
:1009140021838BF31188BFF36F8F03BB002D33D179
:1009240016B120462049B0474FF02003EFF3118B56
:1009340083F31188BFF36F8F238B23F00803238382
:10094400238BDA0628D5012123F010032383B4F87E
:10095400189009F0070900297FF45BAF51E7A168FB
:100964000029DBD00B68002B38BF00239946524680
:100974003B462046D1F804B0D847B9F1000FCDD09A
:100984004946D9F80030EEE729463B465246204610
:100994002D6802F0E4FDC1E713F020011EBF23F02F
:1009A400200302212383D2E78F3500004FF0200378
:1009B400EFF3118183F31188BFF36F8F0123094A89
:1009C400C2F8003502F55B52103253631360C2F86B
:1009D4003432C2F8303481F31188BFF36F8F0020B2
:1009E400704700BF0010005048B1054B1A68054B12
:1009F400B2FBF3F2044B504343F001031847704732
:100A04003C00002040420F0090420000044608B51C
:100A14004FF02002EFF3118382F31188BFF36F8F3D
:100A240002F0D2FF204600F075FD034802F06EFD8F
:100A340000F012FCFCE700BF3844000010B5074882
:100A440001F026FC064C074B1860204600F024FFFA
:100A54002046FFF783FD002010BD00BF6144000065
:100A64006D0A0000680200200A2838B50446074DC4
:100A740004D1286883680D215B68984728688368D7
:100A8400E1B25B689847204638BD00BF6802002089
:100A94000E4A70B5841A05460C20A3100C4C0E4661
:100AA4005C43E4B200FB042040215C3002F0F6FE1B
:100AB400011E05DB074B03EBC40463689847002160
:100AC40028463346BDE87040184700BF7C0200202A
:100AD400B76DDBB6AC4200002DE9F0410C25104E99
:100AE4008046841BA3100F4C0F465C43E4B265435D
:100AF40005F15C004021304402F0E9FE011E09DBEF
:100B0400094A7319C3E91527084B53F83430BDE873
:100B1400F041184740463B46BDE8F041184700BF46
:100B24007C020020B76DDBB635390000AC42000012
:100B340001460C2300224B43084870B5C4185C33AB
:100B4400D4E915561844626502F0DFFE2DB1324631
:100B54002B46BDE870400248184770BD7C02002057
:100B6400A800002010B1012804D07047034BDB6DAE
:100B74005B0701D1FFF7DCBF704700BF7C02002098
:100B8400094B0A4900F01F024009012808BF0B461F
:100B940003EB8203D3F8002222F0E04242F04052F9
:100BA400C3F80022704700BF0025845000288450F9
:100BB4002DE9F843002201210646052000F0FAFA47
:100BC400052000F0D9FA0020FFF7DAFF0120FFF733
:100BD400D7FF114801F0F4F9104B984219D103F0F2
:100BE400B6F800244FF01C080C27DFF83490F568A1
:100BF400494608FB045002F0E5FC002807DB01230A
:100C040007FB04551C44032CEB65F0D10020BDE820
:100C1400F8836FF00400FAE7690B00000000AD0BE5
:100C2400C442000008B54FF02003EFF3118183F3B1
:100C34001188BFF36F8F124A136843F0020013F058
:100C4400010310600CD04FF05022D2F80C34D2F8CB
:100C54000C2413F0010303D00A4802F056FE0123CA
:100C640081F31188BFF36F8F23B1BDE808400020E2
:100C7400FFF75EBF0120BDE8084001F0B1B900BF35
:100C8400F4020020D8020020074BD3E8EF2F22F013
:100C94000201C3E8E01F0028F7D1D30702D40120E2
:100CA40001F0F2B9704700BFF402002000230122D2
:100CB40010B588B0CDE906320193094B04AC01AA02
:100CC400CDE90444CDE9023402F05EFE002805DBE0
:100CD4004FF480420023204602F0A2F808B010BD71
:100CE400473900002DE9F843012206463949D1E885
:100CF400EF3FC1E8E02F0028F9D133B9364937482E
:100D04004B60CB608A6002F070FC731E012B32D8FA
:100D1400012E07D14FF05023D3F81C3403F0030302
:100D2400022B28D003F00EF9044618B92C4B1B787B
:100D3400002B47D14FF02003EFF3118583F3118883
:100D4400BFF36F8F0124274FDFF89C80DFF89C905E
:100D54004FF05022D2F81834D2F81824D2030CD50C
:100D640003F00303022B01D0012E06D124B385F333
:100D74001188BFF36F8FBDE8F883C4B1284600F033
:100D840079FA4FF05022D2F81835DBB2012BDFD1BB
:100D940039680029DCD00021396039680221C2F8A1
:100DA40018152022C8F88021C9F80030D0E70021A6
:100DB400212001F0EFFFE4E74FF050230222C3F8B3
:100DC4000423D8E74FF0502302220546C3F8082332
:100DD400B9E700BFF80200206C020020980200204E
:100DE400CE0800200451005000E100E008500050FB
:100DF400821C084B22F07F42C3F84025D3F8042517
:100E0400904200D17047D3F80405821C22F07F423F
:100E1400F2E700BF005001500022074B1A601B6824
:100E2400064A074BD3F840051368C01A20F07F40E8
:100E34000344136002F080B940510150FC020020C9
:100E44000050015038B500244FF400120E4D0F4BE2
:100E5400C5F808451C601B680D4B0121C3F88021AF
:100E64004FF480332246C5F80433152000F0A2F96C
:100E7400152000F081F90123064A022013602B603B
:100E8400FFF730FF204638BD00500150405101505B
:100E940000E100E008500150F8B52D4B2D4CD3F87B
:100EA40004252D4BB0F1FF3F08BF20461968521AA4
:100EB40022F07F43120238D4013820EAE070A042C5
:100EC400A8BF204601331844A04294BF0C180C1943
:100ED4004FF4803000261E4A204DC2F80803D2F891
:100EE4000415D2F840352E605B1A23F07F432F6837
:100EF400012B21F07F47C2F84075C2F8440304D1A6
:100F04000F2003F025F82E602B684FF40012144BC9
:100F1400C3F880210E4BD3F80405221A22F07F4235
:100F2400012A04D1FFF764FF0BE00020CAE724F094
:100F34007F42C3F84025D3F80405241A023C230257
:100F4400F0D44FF48032024BC3F80423F8BD00BF41
:100F540000500150FFFF7F00FC020020405101506F
:100F640000E100E04FF02002EFF3118382F31188D7
:100F7400BFF36F8F064AD2F80405064A1268801A36
:100F840020F07F4083F31188BFF36F8F704700BF59
:100F940000500150FC020020014802F097B900BF44
:100FA400D042000008B530B143683BB1006801F09D
:100FB4006FFB002008BD6FF4E040FBE70048F9E751
:100FC400EA8FFFFF10B5044618B90B4B0B485B685A
:100FD4009847616859B111F00201206808D00146B0
:100FE400074801F0B3FA002323600023636010BDB7
:100FF400142202F062FDF8E7480000207844000063
:101004000003002010B5044618B9144B14485B685B
:1010140098476368CBB92368BBB94FF0FF324FF0F0
:10102400FF3321460F4801F05FFA08B923681BB962
:101034000A4B0D485B68984714220021206802F08F
:101044003CFD636843F002036360206802F0C7FE5E
:10105400636843F00103636010BD00BF48000020D3
:1010640078440000000300209E44000008B568B1E5
:10107400436873B100684FF0FF334FF0FF3201F063
:101084008FFA054B002818BF184608BD6FF4E040DE
:10109400FBE70248F9E700BFE98FFFFFEA8FFFFF94
:1010A40008B5064940231422054802F07DFEBDE838
:1010B40008400449044802F05BB900BF1C03002047
:1010C40000030020E8420000D8420000094A0A490F
:1010D400936809689867D96708494B6843F0805357
:1010E4004B60002383F31188BFF36F8F9368D86F2D
:1010F400704700BF740800209043000000ED00E03A
:1011040013498A684FF038001044EFF3098C80E8E3
:10111400F01F202080F31188BFF36F8F0D4F4FF025
:1011240000664A6A8A603E60906F0023936780F38A
:10113400118802F1380090E8F01F8CF3098802F15D
:10114400000004B502F048FCBDE80440704700000C
:101154007408002004ED00E01EF0040F0CBFEFF350
:101164000880EFF30980816911F8021C0229FFD07D
:1011740001B502F037FC01BD43B2002B08DB0122AC
:1011840000F01F0002FA00F0024A5B0942F8230053
:10119400704700BF00E100E0054B420953F82220EC
:1011A400012300F01F0003FA00F01040704700BF55
:1011B40000E100E043B2002B01F10101ACBF03F1F7
:1011C4006043064B4FEA4111C9B2ABBF03F561431B
:1011D40000F00F0083F800131954704714ED00E079
:1011E40042F8203C009B0B4942F81C3C019B21F037
:1011F400010142F8183C029B42F8081C42F8143CD6
:101204004FF0807342F8043C0023203A82658367E0
:10121400704700BF81360000044608B50E461546E7
:1012240000F0C2F9084B9C60A36E83F30B88284638
:1012340086F30988002163B681F31188BFF36F8FA9
:101244000022002302F01AFA740800200149102237
:101254000A60704710ED00E072B6404080F31188D8
:10126400BFF36F8FBFF34F8F30BF62B6BFF36F8F83
:10127400704700BF72B6494081F3118820BF80F3E4
:10128400118862B6704700BF30BFFFF7FDBF00BFD3
:101294000E4A08B50E4B22F07F029A60BFF34F8FBF
:1012A400BFF36F8FD3F8882022F47002C3F888202C
:1012B400EFF3148323F0040383F3148801F02AF872
:1012C40001F032F800F038F901F06CF80000000089
:1012D40000ED00E001B572B60B4A106A00281EBF8B
:1012E4000021116202F05EFD62B6EFF30580A0F109
:1012F40010004FEAC0000549014409C99847BDE8F8
:101304000140034908470000740800205C400000C5
:10131400FD14000002F099FA202080F31188084897
:101324004FF40061401880F30988EFF31480022120
:10133400084380F31488BFF36F8FFFF7A9FF000001
:10134400100E0020EFF30880EFF3098101B5724617
:1013540000F052F801BD00BF0C4B9A6A9A6A9A6A6F
:10136400920708D55A6B9A6A120604D518B19A6A7C
:1013740022F080029A620020044B9A6A9A6A9A6A5E
:101384009A6A42F0FF029A620870704700ED00E02A
:101394000D4B9A6A9A6A9A6A920508D59A6B9A6A68
:1013A400120404D518B19A6A22F400429A62002009
:1013B400054B9A6A9A6AD20558BF9A6A9A6A42F4A5
:1013C4007F429A620870704700ED00E0094B9A6A08
:1013D4009A6A986A9A6A9A6A9A6A9A6A9A6A10F4EB
:1013E40080106FEA02426FEA124218BF02209A622A
:1013F400704700BF00ED00E070B5364B0E465B68E9
:1014040000258AB0C3F3080385F31188BFF36F8FF7
:1014140002F07F41B1F17F4F11D102F00C01082994
:101424000DD0110701D4064601250022033B8DF897
:101434000720032B47D8DFE803F0043E423B2E4647
:10144400F3E7244BDA6A92073DD4DC6A14F0804453
:1014540008D028331B78EBB101200DF10701FFF709
:101464007BFF04469DF8073093B92022314602A839
:1014740002F0F8FA099B45B3C3F3080222B96FEAF4
:1014840053236FEA43230993204602A902F0A8FAE2
:101494000AB070BD104B1B782BB101200DF1070170
:1014A400FFF776FFDDE70D4B188884B2002CD9D006
:1014B400FFF78CFFD5E700200DF10701CFE70020EF
:1014C4000DF10701ECE70024CCE723F4FF7323F0CC
:1014D4000103D8E700ED00E029ED00E02AED00E08B
:1014E400044B5A6942F010025A615A6942F480620C
:1014F4005A61704700ED00E0044B9968586A8842CD
:1015040003D003494FF080520A60704774080020EA
:1015140004ED00E0BFF34F8F0549064BCA6802F49F
:10152400E0621343CB60BFF34F8F00BFFDE700BF02
:1015340000ED00E00400FA05002320210348C2184E
:101544000133452B82F80013F9D1704700E100E024
:1015540010B5044601F0A2FA114B9B68A34207D1CF
:10156400EFF3058383B10F4A536843F0805353600C
:101574004FF02003EFF3118083F31188BFF36F8FD3
:10158400BDE8104002F032BC4FF02003EFF31180AD
:1015940083F31188BFF36F8FFFF798FDE8E700BF6F
:1015A4007408002000ED00E010B50E4B88B00293E3
:1015B4000D4B0E4C03930E4B0E4A049302AB019356
:1015C40001A82346012100F007F9002307930A4BE1
:1015D4000121E41A05A80593069400F007F908B060
:1015E40010BD00BF00000020000000000000072024
:1015F40006000100000000206001002010B50B6807
:101604000C7A23F01F0204F01F031A43CB68640909
:1016140023F01F03044943EA440343F001038860B1
:10162400CA600B6110BD00BF90ED00E02DE9F04FE2
:1016340007468846144600264A4D85B046450BDACF
:1016440057F82630D3F80490B9F1000F3AD0B9F125
:101654001F0F05D86FF01504204605B0BDE8F08FC4
:1016640019F01F0FF6D1D3F800A01AF01F0FF1D113
:10167400504602F0E2F9834609EB0A00013802F011
:10168400DCF98345E6D11BF1160FE3D0631E5B45FD
:10169400E0DBC5F808B0E868C5F808B02B6957F86E
:1016A400261020F01F0043F01F0AD1E900321A442B
:1016B400984202F1FF3918D1CA4505D15FFA8BF07F
:1016C40002F09BF90136B9E7C5F808B0EB6822F0DF
:1016D4001F0203F01F031A43EA60E0B202F08DF91F
:1016E40010F1160FB6D0441CECE7C5F808B02A690F
:1016F400013B23F01F0302F01F021343CA45E0B26B
:101704002B61EBD002F079F910F1160FA2D0C5F8D5
:1017140008B0EA689DF808300AF1FF3A62F304035E
:101724008DF808302B699DF808205B0863F3471295
:1017340057F826308DF80820D3E900130B440093A2
:1017440023F01F0301305344A3EB0903C0B223F079
:101754001F03072803933FF67DAF6946FFF74EFF4B
:10176400C1E700BF90ED00E00522034B5A60BFF3D0
:101774004F8FBFF36F8F704790ED00E0BFF35F8F23
:101784000022014B5A60704790ED00E038B50E4CD2
:101794002568082D14D8FFF7F1FF00200B4B0C4AE5
:1017A4001A63854205D10B4B1D70FFF7DDFF002046
:1017B40038BD616801EB0011FFF720FF0130F0E74D
:1017C4004FF0FF30F4E700BFFC42000090ED00E072
:1017D400AAFF4400CC08002010B5034C2278FFF780
:1017E40025FF207010BD00BFCC0800202DE9F74F65
:1017F400264D8A4606464FF00008AB46244FD04596
:101804001BDAD6F80490B9F1000F39D031680846D4
:10181400019102F012F90199044609EB0100013823
:1018240002F00BF984424FF014021A4B08D06FF007
:10183400150302FB08F84BF8083003B0BDE8F08F3D
:1018440014F1160F2C60F8D01978A142F5DD02FBD3
:1018540008B0BC60BC60FC6800F10801007B64F364
:101864000400087138690C79400860F347140C715E
:10187400F96821F01F016960396921F01F012961AC
:1018840008F1010814350C36B9E700BF1C08002024
:1018940090ED00E0CC080020014B1860704700BFB9
:1018A4002400002008B5094B1A786AB901210D20DB
:1018B40019700521FFF77EFC0D20FFF75DFC4FF04A
:1018C4000042034BC3F80423002008BDCD080020C8
:1018D40000D000502A4BF0B544682A481340834294
:1018E4003FD00DD8062B15D005D89BB1022B3AD08A
:1018F4006FF0150034E0B3F5801FF9D1012309E03E
:101904002148834231D0B3F5A00F30D0B3F5800F16
:10191400EED10223D0064CBF0326C2F3401682F454
:1019240080759705C2F34020C5F3002506D512F44F
:10193400006F67681DD001228A40BA60277A134A73
:10194400134C01F01F01012F08BF144640EA450261
:10195400002042EA032343EA8603803144F821301D
:10196400F0BD0723D6E70423D4E70523D2E70323F6
:10197400D0E7520542BF01228A40FA60DEE700BF89
:101984000600F00006001000020040000028845009
:101994000025845010B5094B094C00F01F02400982
:1019A400012808BF234603EB8203D3F8002222F464
:1019B400403242EA0142C3F8002210BD002584509F
:1019C40000288450F8B50D464168C768087A05F0C8
:1019D4001F06B2F5A03F46EA401611D16B4CDFF862
:1019E400B8C17009012814BF2046604606F01F01E3
:1019F400803150F82110CC0707D56FF02200B7E0F2
:101A0400B2F5005FF96800F0A4800121F868A940EC
:101A14000143F96001217869A940B2F5A03FBA6990
:101A24000CBF08438843B3F5C02F0CBF0A438A4355
:101A3400B3F5802F4FF00003BA613A6978610CBFA7
:101A4400114322EA0101524A3961D2F80413C9B29E
:101A540003F5A27052F82000C0F3052086427DD120
:101A640021FA03F0C00779D501219940CC434948B4
:101A7400D0E8EFCF0CEA040CC0E8EECFBEF1000FC3
:101A8400F6D19B0003F1A04303F55043D3F81005AE
:101A940020F00100C3F81005C2F8081300213046F5
:101AA400FFF778FFFB68EB4013F001034FD07B692D
:101AB400EB4013F001045CD0BB690022EB40DB0770
:101AC40054BF396903254FF001075EBF21FA05F5BC
:101AD40005F00105C5F102052E4958BFEDB207FA1C
:101AE40002F4D1E8EF0F40EA0403C1E8EC3FBCF193
:101AF400000FF6D1D04010F0010334D1910001F170
:101B0400A04101F55041D1F81005403220F44F3086
:101B140020F44070C1F8100536029200D1F8100587
:101B240006F47C5692B246EA054602F1A04202F55A
:101B340050420643C1F8106513601268D1F81025AD
:101B440042F00102C1F81025114AC2F804431846B4
:101B54000EE00120A84021EA00015AE70133082BD6
:101B64007FF476AF9AE70132082AB8D16FF01200F9
:101B7400F8BD39693046E94001F00101C1F10301C2
:101B8400C9B2FFF707FF2046F2E700BF00258450E3
:101B940000D000506808002000288450F7B50026C3
:101BA400CDE90066264D2C684CB1264802F00EF8AB
:101BB4000090254802F00AF801902E602B6800225C
:101BC40001269446214DD5F8043306FA02F1194250
:101BD4001BD0910001F1A04101F551410B68A3B163
:101BE40002F5A27355F8233002AFC3F3403007EB7C
:101BF400800050F8087CC3F3042306FA03F33B4344
:101C0400C1F800C040F8083C0B680132082ADAD158
:101C1400009A1AB10B490E4801F075FF019A1AB1E6
:101C240009490C4801F06FFF44B1064801F0F6FF82
:101C3400054803B0BDE8F04001F0F0BF03B0F0BDCB
:101C44007CD10050D8000020E800002000D00050D3
:101C54003408002050080020F0B54B79012B2BD01C
:101C6400032B26D110278B79032B22D1CD7925B1D3
:101C7400012D1ED143681B79DBB10A79012A1DD0DD
:101C8400022A1FD0AAB914460B684668B3F5164F4A
:101C940036686ED033D8B3F5165F6DD01CD8B3F563
:101CA400966F6BD010D8B3F5967F6AD0B3F5167FD4
:101CB4006AD06FF022005BE00027D4E74FF4807411
:101CC4000E22E1E70024FBE7B3F5166F5FD0B3F50E
:101CD400965FEED1384B3EE0B3F5E14F5AD007D8CA
:101CE400B3F5615F58D0B3F5964FE2D1334B32E090
:101CF40047F6122C6345DCD14FF400032BE0B3F517
:101D0400613F4BD013D8B3F5963F4AD009D84DF66E
:101D1400C02C634547D0B3F5614FCAD14FF46B0370
:101D240019E0B3F5E13FC4D14FF0EB7313E0B3F521
:101D3400612F3BD009D8DFF898C0634539D0B3F59B
:101D4400E12FB6D14FF0E86305E0DFF888C06345C2
:101D5400AFD14FF08053C6F82435C3682C433A43BF
:101D64002243043303C9C6F86C2583E8030000202A
:101D7400F0BD4FF41D03EEE7114BECE74FF49E2347
:101D8400E9E74FF4A033E6E74FF41C33E3E74FF4FD
:101D94001D23E0E70B4BDEE70B4BDCE74FF06C73E6
:101DA400D9E70A4BD7E74FF46503D4E74FF07063E4
:101DB400D1E74FF08063CEE700B0130000A04E00DF
:101DC4000050270000C0750000F03A0000903A016E
:101DD40090D0030040420F00074B084900F01F0257
:101DE4004009012814BF1846084602F18003032263
:101DF40040F82320704700BF0025845000288450F9
:101E0400064B074900F01F024009012814BF184679
:101E14000846012393408360704700BF0025845027
:101E240000288450F8B500274368C6681C68054636
:101E3400C4F8007530601420FFF7E2FF1420FFF7A8
:101E4400CBFF1422154B1320C3F85872C4F80C2589
:101E54001622C4F81425C3F85472FFF7D1FF1320D7
:101E6400FFF7BAFF1323C4F808351523E968284699
:101E7400C4F810350431FFF7EFFE68B90823C4F83D
:101E84000035C4F81001D4F8103101231036C4F819
:101E94003465C4F838352360F8BD00BF002584508C
:101EA400054B1868043B1B68072B03D1831E58425B
:101EB40058417047002070473401FF004FF0502311
:101EC400D3F85825034B02F00302D340024A1360AF
:101ED400704700BF0020A1073C00002008B5FFF7B1
:101EE400DFFF48B1304B1A6832B90D211960012166
:101EF400A3F5827319601A600022D30003F57F03EF
:101F0400D3F80013013107D0D3F800130132D3F80A
:101F14000433202A0B60F0D1FFF7C2FF00283CD124
:101F2400FFF7BEFF38B1214B214A1A604FF050230E
:101F34000122C3F85825FFF7B3FF10B100221D4B4F
:101F44001A60FFF7ADFF50B14FF05023D3F80024CF
:101F5400D10742BF0022C3F81421C3F81821FFF7A8
:101F64009FFF48B14FF05023D3F80024D20744BF59
:101F74006FF00102C3F80024FFF792FF10B165224D
:101F84000D4B1A600D4AD2F88C3043F44063C2F80A
:101F94008C30BDE80840FFF791BF2922064B1A6038
:101FA40003221A63BCE700BF204A00503095035057
:101FB4004400EFBE4C2503500C47005000ED00E0F8
:101FC400044B1A7922B9012218601A710248704729
:101FD400024870476C0800200000AD0B0C00AD0BEC
:101FE400032847D8DFE800F002222D3A4FF05022B0
:101FF400D2F81834D2F81814C90311D503F0030326
:10200400022B0DD1C2F8183500221B4B1A601B6835
:1020140002224FF05023C3F8042301229A60704730
:102024004FF050230122C3F81825EDE70022134B8B
:102034001A601B6801224FF05023C3F804231A606E
:10204400704700220E4B1A601B684FF400724FF069
:102054005023C3F8042301221A6270470022094B5B
:102064001A601B684FF480724FF05023C3F80423A6
:1020740001229A61704700BF045100500051005082
:10208400245100502051005070B5044603283ED816
:10209400DFE800F002223E4B4FF050230222C3F847
:1020A4000823002203F582731A601B68284B01225F
:1020B40042F210754FF050261A60022C42D0032CC5
:1020C40043D024BBD6F81834DB0320D5012001F01B
:1020D4003CFE013DF1D11AE001234FF050240021D0
:1020E40042F210751B4AC4F80833116012681A4A88
:1020F4001360D4F80C34D4F80C2403F00103D20395
:1021040005D523B1012001F020FE013DF1D170BDC0
:102114004FF050234FF40072C3F80823002203F554
:1021240092731A601B680D4BC1E74FF050234FF4B4
:102134008072C3F80823002203F590731A601B68A9
:10214400074BB4E7D6F85C34BEE7D6F85434BBE7A3
:102154000C500050005100500450005024500050C6
:102164001C500050264B10B51A6852B1002018605C
:102174001B6801224FF05023C3F80823214B1B682E
:102184009847214B1A688AB100221A601B684FF0E5
:102194005023D3F81824D3F8181402F00302012AA8
:1021A4004FF0020124D1C3F818159A60174B1A682E
:1021B40062B100221A601B684FF480724FF0502302
:1021C400C3F808230F4B04201B689847104B1A6868
:1021D400AAB1BDE8104000221A601B684FF40072D7
:1021E4004FF05023C3F80823064B05201B681847FB
:1021F400C3F80813034B01201B689847D6E710BDAA
:10220400005100506C08002004510050205100502F
:1022140024510050F8B5104B104F53F820500130A2
:1022240053F82060AE4200D8F8BDD5E9003420460A
:10223400984770B16CB10123E41B094A2411610968
:1022440052F8210004F01F0403FA04F4044342F892
:1022540021400835E6E700BF7C430000A8000020C9
:1022640008010020084BC01A0011084B420953F81A
:102274002220012300F01F0003FA00F010420CBFDB
:1022840018460020704700BFA80000200801002065
:10229400114970B505460E46104C8C4204D10F4CC2
:1022A400B4420AD1002414E02046FFF7DBFF10B14A
:1022B4002368AB420DD01034EFE72046FFF7D2FF7E
:1022C40008B91034ECE72846216801F0BFFB002868
:1022D400F7D1204670BD00BF08010020A8000020EF
:1022E40008B50B4D4FF02002EFF3118382F31188F0
:1022F400BFF36F8F01F044FE012104460228D8BFCA
:10230400084601F04DFE2C62FEF7A6FFEAE700BF87
:10231400740800200248034A0021121A01F0CDBBC0
:1023240060010020D008002008B50648064A074985
:10233400121A01F097FBBDE80840054A0549064812
:1023440001F090BB000000205C0100202445000047
:10235400000000002445000000000020012208B510
:102364000B4B02201A70FFF755FF0A4A0A490B4823
:1023740001F0CCF80320FFF74DFF00F0ABFDFEF7B2
:1023840065F8074A137B23F00103137308BD00BFEC
:10239400CE0800201E450000EC440000F844000074
:1023A400E00100202DE98048344BA7B003F5006913
:1023B40089F3088883F30A880024E023304D4FF022
:1023C400010B85F82230EC772C766C76AC766B6A50
:1023D4002C4E43F4E0236B62FFF782F8FEF736FFDE
:1023E4004FF0FF33AB62EB6240F20113264DADF8C0
:1023F400243006ABAB602046CDE92044FFF70AFF4A
:102404000120FFF707FFDFF898A000F069FC1F4BDD
:102414006E624FF480621E49059330465346CDE9FF
:10242400034BCDE90144009400F024FD737B804606
:1024340023F004033046737301F004FD0F23154F9A
:102444004FF4A072CDE902431349144B3846CDE949
:1024540004B4CDE9004400F00DFD7B7B524623F02B
:1024640004037B7305F1180341463046C5E906337E
:10247400EF602C75C5F80490FEF7CEFE100E002018
:1024840000ED00E0E0010020740800201F4500007A
:10249400D008002060010020D00C0020E5220000BC
:1024A4006123000070B50E4B0E4CA34201D30020F3
:1024B40070BDD3E9030141EA000212F003020BD11B
:1024C4009D685A61AA4201D11C33EEE75E6901326C
:1024D4000E6059610144F5E76FF01500E8E700BFAD
:1024E4000C0100200C010020D3B50C4616461F46F3
:1024F4004FF02003EFF3118183F31188BFF36F8F43
:1025040043695BB123601B68436183690133836161
:10251400002081F31188BFF36F8F11E056EA0702A0
:1025240003D16FF00B002360F3E70246CDE90067A7
:10253400044800F04FFB18B9034B9B685B692360A8
:1025440002B0D0BDCF0800207408002070B5044646
:102554000D464FF02003EFF3118683F31188BFF388
:102564006F8F01F0CAFC58B100212A68C16742612B
:1025740001F068FC3146BDE87040084800F010B92D
:102584002B6862691A602B686361A369013BA361CC
:1025940086F31188BFF36F8F70BD00BFCF08002092
:1025A4002DE9F341044616461F464FF02003EFF38E
:1025B400118883F31188BFF36F8FC368324A6BB1FC
:1025C40080689168884219D056EA070318D188F3C5
:1025D4001188BFF36F8F6FF00F000CE0916891F9D1
:1025E4000E100133E36093682161A36088F31188BE
:1025F400BFF36F8F002002B0BDE8F0812169F0E7DE
:1026040090F90E3091F90E109942A8BF194621EAAB
:10261400E17199422CDA00F01FFB0546224641463F
:10262400CDE90067194800F0D5FA0028E3D04FF04F
:102634002003EFF3118683F31188BFF36F8F2368B0
:102644002169A34207D033B193F90E309942A8BF50
:10265400194621EAE171A06890F90E30994209D136
:102664006DB13146094800F09BF86FF00A00C2E7EB
:102674000025D3E700F0F0FA0028F2D1F0E786F362
:102684001188BFF36F8FF0E774080020CF08002093
:1026940038B583680446002B36D01E4A92689342AC
:1026A40035D1DA7B013ADA73C368012B05D0013BDB
:1026B400C36000F0D5F8002038BD4FF02003EFF3DD
:1026C400118583F31188BFF36F8F0169806890F9D6
:1026D4000E30994201D000F0BFFA204601F00DFC03
:1026E400A06058B190F90E2022610022C26701F067
:1026F400A9FB2946084800F053F8DAE7E06085F3BF
:102704001188BFF36F8FD4E76FF01500D4E74FF053
:10271400FF30D1E774080020CF08002010B5084C22
:1027240023685BB1FEF71EFC03462068054A034498
:102734000021BDE81040136101F032BC10BD00BFA0
:10274400AC08002074080020F8B505460C464FF08C
:102754002003EFF3118683F31188BFF36F8F0022F8
:102764004FF4004740F2E73000210A4BE7FB050134
:102774001A614FF47A720023FDF7EAFC064B1860E5
:10278400064B1C60FFF7CAFF86F31188BFF36F8FF7
:10279400F8BD00BF74080020AC080020A808002081
:1027A40049B9EFF3058030B9054B5A6A9B689A42E0
:1027B40001D0FEF78BBC81F31188BFF36F8F704794
:1027C400740800204FF02003EFF3118183F3118884
:1027D400BFF36F8F044B9A68D37B013BD37381F3B0
:1027E4001188BFF36F8F704774080020094B03F101
:1027F4002802824205D19B688B4202D14B7BDB06C7
:1028040006D1D1E9003213605A600023C1E90033D4
:10281400704700BF7408002070B5104C064604F1E0
:10282400280001F005FB0546A368597B880644BFD0
:1028340041F00801597305B9E5684EB95A7BD206CF
:1028440006D1AA6922B9DA897F2A01D9636270BDE7
:10285400AB4201D0FFF762FF6562F8E7740800201D
:1028640010B54FF02003EFF3118483F31188BFF305
:102874006F8F084B00209A68D37B0133D373FFF723
:10288400CBFF84F31188BFF36F8FBDE8104001F0D4
:10289400B9BA00BF7408002070B4437BDB062AD1A8
:1028A400836943BB154A114651F8284F8C4218BF1F
:1028B4002346002B38BF0023D46AB3B190F90E60CD
:1028C40093F90E50AE4203DBA3420ED01B68F4E72B
:1028D4005A68C0E9003210605860437B63F07F039C
:1028E400437370BC0020FFF797BFC0E90014D36A9C
:1028F4001860D062F1E770BC704700BF7408002014
:1029040010B54FF02002EFF3118482F31188BFF366
:102914006F8F427B510704D484F31188BFF36F8F08
:1029240010BD22F004024273FFF7B6FF2146BDE852
:1029340010400148FFF734BFCF08002070B590F96C
:102944000D300146002B02DA1748FFF74FFF174AF4
:10295400104650F8283FD46A834208BF0023002B56
:1029640038BF0023D3B191F90E6093F90E50AE42F3
:1029740003DBA34212D01B68F4E75868C1E90030B6
:10298400016059604B7B906863F07F034B73431A7B
:1029940058425841BDE87040FFF73EBFC1E900040A
:1029A400D36A1960D162EDE79C0800207408002006
:1029B400014670B54FF02003EFF3118483F31188BF
:1029C400BFF36F8F164B174A98681568A8421D46C7
:1029D40006D1FFF7A3FE84F31188BFF36F8F70BD98
:1029E40000261660104A1268BAB1C2897F2A14D828
:1029F400427BD20611D10D4A90F90E6012689642BC
:102A04000BDB0B4A904208D01A698A4202DCFFF7BA
:102A140095FFDEE7521A1A61DDE700232B61DAE73E
:102A240074080020A4080020AC080020A808002096
:102A34006001002070B50446183001F08BFA4FF0A5
:102A44002003EFF3118683F31188BFF36F8F94F99A
:102A54000D30002B07DA21460E48FFF7C7FE637BD3
:102A640003F07F0363730C4D637BA86843F010038A
:102A74006373031B58425841FFF7CEFE86F3118857
:102A8400BFF36F8FAB68A34203D1BDE8704001F080
:102A9400B9B970BD9C08002074080020036E2DE9AC
:102AA400F041044603B1984704F1180001F052FACA
:102AB4004FF02003EFF3118683F31188BFF36F8F78
:102AC400637BD80623D1A2690ABB190607D5214620
:102AD4001E48FFF78BFE637B03F07F0363731C4B7D
:102AE4009868021B50425041FFF796FE0027637B13
:102AF40004F1300843F008036373256B454500D0A7
:102B040095B986F31188BFF36F8FBDE8F0819B07F9
:102B1400ECD52146A068FFF769FE637B23F002032E
:102B240063730023A360E1E705F1180001F012FAD2
:102B3400A8682946FFF75AFE6B7B284623F0020358
:102B44006B73AF60EF67FFF7A7FED6E79C08002022
:102B54007408002008B590F90D300146002B06DA00
:102B64000748FFF743FE4B7B03F07F034B73054B92
:102B74009868431A58425841BDE80840FFF74CBED4
:102B84009C080020740800202DE9F04106461446F4
:102B94001D464FF02003EFF3118783F31188BFF331
:102BA4006F8F01F07FF987F31188BFF36F8F6B1C70
:102BB40008BFB4F1FF3F08D022462B4606F11800A7
:102BC4000349BDE8F04100F02FBABDE8F08100BF31
:102BD400693E000010B50C46064B11469868064B3A
:102BE4001860DDE90223FFF7CFFF2046BDE810405F
:102BF400FEF76CBA74080020A4080020F8B5054656
:102C040001F0E8F92C184FF02003EFF3118783F358
:102C14001188BFF36F8F0D4E0D4BB0681860FFF72E
:102C240099FFB0680B492A46EB17183000F0FCF9FD
:102C3400B2683846537B43F010035373FEF746FAE9
:102C440001F0C8F9201A20EAE070F8BD74080020E9
:102C5400A4080020693E00002DE9F04104464FF02D
:102C64002003EFF3118883F31188BFF36F8F437B45
:102C74004EB2DB062ED1856965BB184F214607F19C
:102C84002800FFF7B3FDBB6AFA6A834218BF1D46EA
:102C9400002D38BF0025A673B5B195F90E10B142C9
:102CA40003DCAA4210D02D68F6E76A68C4E9005232
:102CB40014606C600120FFF7AFFD012088F31188D8
:102CC400BFF36F8FBDE8F081C4E90002FB6A1C60AA
:102CD400FC62EFE70020A673F0E700BF7408002051
:102CE4000021044B084603F12802C3E90A22FFF736
:102CF4002BBD00BF74080020F8B5244C244BA268F7
:102D04009A4230D04FF02003EFF3118583F31188FA
:102D1400BFF36F8FA16804F12800FFF767FDA36A72
:102D2400A268834208BF0023002B38BF0023E16A56
:102D34002BB392F90E7093F90E60B74203DB8B420A
:102D44001DD01B68F4E75968C2E900310A605A6073
:102D5400537B012063F07F035373FFF75DFD85F31D
:102D64001188BFF36F8F4FF02003EFF3118083F3CB
:102D74001188BFF36F8FBDE8F840FEF7A7B9C2E929
:102D84000001E36A1A60E262E2E700BF740800200F
:102D9400600100200B46013308BFB0F1FF3F10B5BE
:102DA40006D10B4B9868FFF745FE4FF0FF3010BD7E
:102DB400044648B9FFF7A0FF4FF47A7084FB00344F
:102DC400D80B40EA4440F2E7FFF718FF0446F3E764
:102DD40074080020014B9868704700BF74080020F5
:102DE40038B504464FF02003EFF3118583F31188BF
:102DF400BFF36F8F01F081F848B10022C26701F080
:102E040021F82946BDE838400448FFF7C9BCD4E995
:102E140002329A4218BF0133A360F2E7CF080020C0
:102E240037B514461D464FF02003EFF3118183F3A9
:102E34001188BFF36F8F836843B1013B836081F3D3
:102E44001188BFF36F8F002003B030BD54EA05032F
:102E540006D181F31188BFF36F8F6FF00F00F3E792
:102E64000246CDE900450248FFF7B4FEECE700BF97
:102E7400CF0800202DE9FF4100F13005C0E90C55D1
:102E84000E9D04460573042545730D9DD61D85735B
:102E940000250C9A26F00706C0E90655C0E91A1663
:102EA400C573056702920B9A01EB060801920A9A10
:102EB40000924246FEF794F9054BC4E917559B6806
:102EC40003B15B6F4046636704B0BDE8F08100BFA7
:102ED400740800202DE9F0472A4E2B4DB04686B0E9
:102EE400B54205F1300410D3FFF76CFC4FF40049F0
:102EF40040F2E7360027244CDFF890A0444521D364
:102F040006B0BDE8F047FFF7ABBC54F8043C0593AA
:102F140054F8103C049354F8143C039354F8183CAC
:102F2400029354F81C3C019354F8203C009354E958
:102F34000A2354E90C01FFF79DFF54F8303CDD658A
:102F44002546CDE7636A5A1C0DD03046394623EA3C
:102F5400E373C9FB0301B94208BFB042256804D139
:102F64002846FFF7CDFC3034C8E74FF47A720023CB
:102F7400FDF7EEF802460B4605F11800514600F045
:102F840053F8F0E70C0100200C010020693E00001A
:102F9400034B1B680BB9FDF7E5BF0020704700BF6A
:102FA400B008002030B5036868B10A4A52689042FC
:102FB40009D043B1D3E90421D0E90445121945EB02
:102FC4000101C3E90421426813605A600023C0E987
:102FD400003330BD4000002038B5114B1C689C42C2
:102FE40008BF0024FFF7D4FF0546ACB1D4E90401BF
:102FF400401B61EBE571B0F1004F71F100030BDA96
:10300400002871F1000300DA0020064B1B6913B19C
:103014009842A8BF184638BD6FF00040F5E700BFDE
:1030240040000020740800202DE9F74F0191194653
:103034004B1C08BFB2F1FF3F82466BD06FF0010317
:103044004FF0FF3B541C41F10005B3EB04086BEB5C
:103054000509B8F1000F79F100030FDBFFF798FFC2
:103064006FF00103324AD2E9001C5B1A6BEB0C02CD
:103074001E1B62EB0507341A67EBE075019BCAF867
:1030840008304FF02003EFF3118683F31188BFF368
:103094006F8FFFF77DFF012C75F10003BCBF012486
:1030A4000025244B24181A6845EBE0759A42CAE9B6
:1030B400044501D05F6852B95A68CAF80030CAF8AA
:1030C40004205A68C2F800A0C3F804A014E0D2E9AE
:1030D4000489DAE90445444575EB09011DDAB8EBC6
:1030E400040069EB0501C2E904015168CAE9002141
:1030F400C1F800A0C2F804A01A689A4206D092450A
:1031040004D1FFF769FF0021FDF7C6FE86F311889D
:10311400BFF36F8F03B0BDE8F08FB4EB080065EB2D
:103124000901BA42CAE90401C6D01268C3E700BF64
:1031340060020020400000202DE9F74F0646FFF70B
:1031440037FC4FF02003EFF3118483F31188BFF3AE
:103154006F8FDFF8B0A02A4D5146DFF8ACB02E6077
:10316400D5F800C0DBF800006246DAE90089D3171D
:103174005845CDE900230DD060B1D0E90467B445CA
:10318400BB411DDA009BB6EB030C019B67EB030606
:10319400C0E904C60026009B2E6013EB0802019BC5
:1031A40043EB0903C1E90023FFF716FF3146FDF79E
:1031B40073FE84F31188BFF36F8F03B0BDE8F08F03
:1031C4000022002318EB060849EBE679C0E9042342
:1031D400ACEB0606CAE900892E60FFF7E3FE84F330
:1031E4001188BFF36F8F836898474FF02003EFF384
:1031F400118483F31188BFF36F8F0249B0E700BFD6
:10320400B0080020600200204000002010B54FF0FC
:103214002003EFF3118483F31188BFF36F8FFDF75D
:10322400A1FE064BD3E90023121843F1000384F3F3
:103234001188BFF36F8F1046194610BD600200203D
:1032440038B5064C064DAC4201D3002038BD2046AB
:10325400D4E9011200F0C2FE1434F4E70C0100209A
:103264000C01002010B50A4C23681BB10123002077
:10327400236010BD00F098F80028F7D00138072823
:1032840003D8044B53F8200010BD034810BD00BF01
:10329400B408002094430000FE8FFFFFBFF34F8F5C
:1032A4000549064BCA6802F4E0621343CB60BFF3DE
:1032B4004F8F00BFFDE700BF00ED00E00400FA05FA
:1032C400014B5B68184700BF48000020024BD0E95F
:1032D4000012C3E9001270474800002048B1436857
:1032E4002BB1BFF35F8F0023036018467047024879
:1032F40070476FF4E0407047EA8FFFFF10B5044653
:1033040028B1636813B100232360636010BD024BCE
:1033140002485B689847F4E748000020B443000083
:1033240010B5044630B100226368226043F0010303
:10333400636010BD0148FFF7C3FFF4E7DC430000FE
:1033440080B1436863B10122D0E8EF3FC0E8E12FC8
:103354000029F9D1012BF7D0BFF35F8F002070470C
:10336400024870476FF4E040704700BFEA8FFFFFE8
:1033740070B40B4B0668C268D0E90154C3E9024239
:10338400C3E90065D1E903020E68064BD1E9015493
:10339400C3E90065C3E902401A6170BC704700BF0D
:1033A400580000206800002008B500F00FF828B984
:1033B40000F00EF830B9044A106008BD00F036F889
:1033C400032008BD042008BD0C5A84500020704717
:1033D40010B5114800F048F800B110BD0F4800F0D6
:1033E40043F80028F9D10E4C204600F03DF800289F
:1033F400F3D10C4B0C481C6000F036F80146002851
:10340400EBD100F02DF8044608B1204610BD00F0C1
:103414003FF82046FAE700BFA000002094000020F7
:103424009C000020A40000209800002008B5084853
:1034340000F024F8074800F021F8074800F01EF8CF
:10344400064800F01BF8BDE8084000F00BB800BFC8
:10345400A0000020940000209C0000209800002080
:1034640000207047704700BF08B5034B02681B6813
:1034740010689847002008BD5800002008B5034B89
:1034840002685B6810689847002008BD5800002057
:1034940070B5094C094D2069AB68984718B1084BC1
:1034A40008485B6898470021074AEB681160206967
:1034B400BDE87040184700BF680000205800002095
:1034C4004800002000440000C8080020034658B10A
:1034D400426802F00302012A03D0032A04D10268DD
:1034E40012B10020986070476FF015007047426871
:1034F400034602F00302032A4FF00002816014BF66
:10350400104600685A607047002070470FB407B532
:1035140004A951F8040B0191FDF754F903B05DF8C7
:1035240004EB04B07047038B13F0070305D1036861
:10353400002B0CBF002003207047022B05D1438BC6
:10354400002B14BF002004207047012B05D1036811
:10355400002B0CBF002005207047002070472DE988
:10356400F0410D4607461946281D90461E46FFF7B2
:10357400BEFF044638B13346424629463846A4467F
:10358400BDE8F0416047BDE8F08110B44FF020047D
:10359400EFF3118284F31188BFF36F8F416110BC84
:1035A4000121FDF71DB910B50C4640B139B1081D14
:1035B400FFF78CFF28B9A36833F0030301D06FF041
:1035C400150010BD38B50C46054658B151B10B680D
:1035D40043B14B6833B11C22002100F06EFA002085
:1035E4002C6138BD6FF01500FBE770B504460E463C
:1035F400FFF7D9FF051E31DB4FF02003EFF31181F4
:1036040083F31188BFF36F8F4FF6FF75638B208BA5
:10361400AB4200F007022ED0022A0ED1013363839D
:103624001546012381F31188BFF36F8FB3B10023D3
:1036340031462046FFF793FF10E0830701D0062AA6
:103644000ED100233360636893B9C4E9006615465C
:1036540062B90A4620460221FDF7C2F8284670BD29
:10366400052A0CBF6FF022056FF004050023D9E78B
:103674001E606660EBE76FF00A05F7E7044608B5DD
:10368400084611461A46A047FFF7A4FBFDF760FF62
:10369400836800EBC101B3F5004F2CBF51F8220041
:1036A40031F81200704700EBC1018068B0F5004F9B
:1036B4002CBF41F8223021F812307047012208B59E
:1036C400FFF7E6FF400808BD836800EBC101B3F5CE
:1036D400004F08D34B681AB143F001034B607047A5
:1036E40023F00103FAE74B881AB143F001034B803E
:1036F400704723F00103FAE753000122FFF7D3BF19
:1037040080680131B0F5004F2CBF02200120081A57
:10371400B0FA80F0C0F11F0070472DE9F041044673
:103724000D46FFF7CBFFA3680146B3F5004F01D365
:10373400012835D02046FFF7E3FF04EB8002166929
:103744009EB9012303FA00F0E36829460343E360CA
:10375400204615612B460222FFF7A5FF03222946C6
:103764002046BDE8F041FFF79EBF022231462046C5
:10377400FFF78EFF07460346022229462046FFF73D
:1037840092FF3346032229462046FFF78CFF03228B
:1037940039462B462046FFF786FF02223146DFE7F3
:1037A400BDE8F081B2F5802FF8B52CBF08250425BB
:1037B4000023551B0022CC1D24F007040460C4E937
:1037C400002300230D4425F007052D1BED08294691
:1037D4002046A560E360FFF793FF8600411C18466E
:1037E4001B36F60804F110028B4229DB32462046D0
:1037F4000021FFF781FFAF1B204601220021FFF7C4
:1038040063FF3A463146FFF777FF33463146204699
:103814000022FFF748FF294620460022FFF76CFFED
:103824003B46294620460022FFF73DFF2946204615
:103834000122FFF749FF3146BDE8F840FFF76DBFAD
:1038440042F8040B0133CFE77047FEF747BB4FF450
:103854007F0345F24032D3F80C12914207D1D3F8DA
:10386400100210F1BE3F14BF002001207047002059
:10387400704708B5FFF7EBFF28B1404080F311888B
:103884004FF0040002DF002008BDCBB20C21C26857
:1038940003FB0121C86D00F0070070474FF02003BF
:1038A400EFF3118283F31188BFF36F8F036813F072
:1038B400C00301D08B4207D101230360002082F3AF
:1038C4001188BFF36F8F70474FF0FF30F7E710B5E3
:1038D4004FF02003EFF3118283F31188BFF36F8F4E
:1038E400036803F00704012C06D10160002082F371
:1038F4001188BFF36F8F10BD03F0C0038B4214BF58
:103904004FF0FF306FF00F00F1E74FF02003EFF3BB
:10391400118283F31188BFF36F8F036803F0C00330
:1039240043F00203036082F31188BFF36F8F704783
:1039340010B41C24C068CBB203FB0400002110BCEB
:1039440010471046FFF74CBA0220FEF79DBB00203B
:10395400FEF79ABB0220FEF743BB0020FEF740BBF4
:1039640038B50C23CCB263430546C0685C33802170
:103974001844FFF793FF002805DB696801EBC404D2
:1039840063689847002038BD2DE9F0414FF00C08DA
:10399400CDB208FB05F8C468064608F15C00802136
:1039A40020441746FFF793FF002809DB7B68444453
:1039B4006365BB68A365736853F835309847002086
:1039C400BDE8F0817047704770470020FDF71EB8CE
:1039D4000021012000F004B8836E83F30B88704744
:1039E40000F0C5B90146006800F0C1B908B5FDF79B
:1039F4004BFCBDE80840FDF77FBD30B54B680C6853
:103A040085B00A898D7A0094013B24F01F04234475
:103A140002F01F0242EA451223F01F03072804465E
:103A24008DF80820039305D86946FDF7E7FD204685
:103A340005B030BD6FF01504F9E740E800F313F466
:103A4400803FD8B208BF6FF015007047431E01399C
:103A540013F8012F11F8010F824201D1002AF7D186
:103A6400101A7047F0B581EA0004A50703460BD08D
:103A7400013B0A4491421BD1F0BD002AFCD011F84D
:103A8400014B013A03F8014B9C07F6D122F00304E1
:103A94001D1F96080F19B94205D16FF00305234481
:103AA40005FB0622E4E751F804CB45F804CFF2E71E
:103AB40011F8014B03F8014FDCE7034670B5C9B2B6
:103AC4009C0711D141EA012422F0030644EA04458B
:103AD4001E449408B3420DD16FF0030505FB042284
:103AE4001A44934209D170BD002AFCD003F8011B8B
:103AF400013AE5E743F8045BECE703F8011BF0E760
:103B04004FF0FF30704770B50E460168154689B115
:103B14000C68002C38BF00248A682A4002D0304642
:103B24004B68984734B123682146002B38BF0023E3
:103B34001C46F1E770BD436800205B681B690B609D
:103B4400704743685B68586842400A4042405A6084
:103B540000207047436800205B68996070474368A1
:103B640000205B68D9607047436800205A68536836
:103B74004B4053607047C36830B5586858B100244F
:103B8400814213D108685CB99C685860A14200D195
:103B940098600020086072B9002030BD2846EFE725
:103BA40020609868814208BF9C60F2E7056804467B
:103BB400002DF3D13AB15A680A6098685960002818
:103BC400EAD19960E9E76FF01500E6E72DE9F041E5
:103BD40001260027C368D0F80480DC68D3E90521F6
:103BE4000A4324EA0204D8F804201B6915695D40DD
:103BF40024EA050514B92846BDE8F08134420AD008
:103C040098F8083007F01F00002140EA4310FDF740
:103C1400C1FE24EA060401377600EBE72DE9F04102
:103C240001260025C768D0F80480FC68D7E905326E
:103C3400134324EA03040CB9BDE8F081264210D0F2
:103C4400396998F80830E94001F00101C1F1030134
:103C540005F01F00C9B240EA4310FDF79BFE24EAB9
:103C6400060401357600E6E70B46C268D2E9010195
:103C740083E803000020704743681B68D3F880047E
:103C8400C3F8800470474368C2681B68D3F8100106
:103C940048B10020127C0A70C3F81001D3F8102137
:103CA40001221A6070474FF0FF3070472DE9F3414D
:103CB40043688DF807101C68C66800F043F998BB88
:103CC40064254FF0010806F10C07D7E8EF3F002BFD
:103CD40003D1C7E8E28F002AF7D107D021200021C1
:103CE400013DFFF757F815F0FF05EED10023C4F8A6
:103CF4002031D4F820310DF10703C4F844350123F1
:103D04004FF47A75C4F84835A360D4F8203123B948
:103D1400012000F01AF8013DF7D10123E3600023EC
:103D2400F36002B0BDE8F0810123F360DEE7002018
:103D340008B5FDF7EFFB08B5FDF72EF9FDF7B0F96F
:103D4400BDE80840FFF78EBA004700F001B908B596
:103D54000520FDF721FA10B90520FDF70DFA4FF003
:103D640050230122C3F81425C3F8802508BDF8B5F3
:103D740005460E464FF02003EFF3118783F31188B5
:103D8400BFF36F8FFFF726F8314604462846FFF746
:103D9400CEFF87F31188BFF36F8F2046BDE8F8404C
:103DA400FDF7D6BBFFF70FBE30B50024846141EAAE
:103DB400020414F00304C0E9023201610CD144612D
:103DC400A34203D1C0E90000002030BD456901349D
:103DD4000D6041611144F3E76FF01500F5E7034608
:103DE4000020C3E90033C3E902007047034620B949
:103DF400EFF305820AB9FDF769B983F31188BFF3BC
:103E04006F8F70474FF02003EFF3118083F3118815
:103E1400BFF36F8FFFF7EABF014608B58068FEF76E
:103E2400E5FC4B7B23F002034B7300238B6008BD3E
:103E340003460068834203D0002838BF002070473F
:103E44000020704710B54FF02003EFF3118483F383
:103E54001188BFF36F8FFEF71FFD84F31188BFF342
:103E64006F8F10BD70B504464FF02003EFF3118639
:103E740083F31188BFF36F8F50F8103CA0F118053D
:103E840013B12846FFF7C8FF14F80B3C284623F06B
:103E9400140304F80B3CFEF7FFFC86F31188BFF310
:103EA4006F8F70BD38B504460D46FEF753FE637B35
:103EB40043F002036373C5B12B68A5609D4208BF3C
:103EC4000023002B38BF002383B194F90E1093F91B
:103ED4000E20914204DB6A689A4207D01B68F3E71C
:103EE4005A68C4E9003214605C6038BD6B682560B0
:103EF40063606B681C606C60F7E738B54FF02003B3
:103F0400EFF3118283F31188BFF36F8FFFF790FFF4
:103F1400044682F31188BFF36F8F88B14FF02003FA
:103F2400EFF3118583F31188BFF36F8FFFF774FFED
:103F340085F31188BFF36F8F04F1180000F00AF8BD
:103F4400204638BDEFF30580003818BF01207047C4
:103F5400FCF74ABD10B54FF02002EFF3118482F351
:103F64001188BFF36F8F03683BB1FFF71BF8002084
:103F740084F31188BFF36F8F10BD6FF01500F7E75E
:103F840010B54FF02003EFF3118483F31188BFF3CE
:103F94006F8FFFF721F884F31188BFF36F8F10BD83
:103FA40070B504460D464FF02003EFF3118683F3FA
:103FB4001188BFF36F8FFFF70FF8012805DDA042CA
:103FC40003DD29462046FCF767FF86F31188BFF31B
:103FD4006F8F70BD08B5FFF719F908BD10B400F173
:0E3FE4000C04C0E9034410BCFFF7DCBB7047BF
:023FF200FFFFCF
:083FF40090C1FF7F01000000F5
:103FFC00B109000000000000A9240000000000002E
:10400C004532000000000000911700000000000085
:10401C00B50B0000A8000020291E0000B8000020ED
:10402C00410A000000000000490E0000C8000020FA
:10403C00A9180000E8000020A9180000D8000020F2
:10404C003B3D0000F8000020773800000000000025
:10405C0000000000D539000000000000D539000038
:10406C0000000000D539000000000000D539000028
:10407C0000000000D5390000692100004D3D000012
:10408C0000000000D539000000000000D539000008
:10409C0000000000D539000000000000D5390000F8
:1040AC0000000000D539000000000000D5390000E8
:1040BC0000000000D539000000000000A11B00002A
:1040CC0000000000D539000000000000D5390000C8
:1040DC0000000000D539000000000000D5390000B8
:1040EC0000000000D539000000000000D5390000A8
:1040FC0000000000D5390000000000001D0E00007B
:10410C0000000000D539000000000000D539000087
:10411C0000000000D539000000000000D539000077
:10412C0000000000D539000000000000D539000067
:10413C0000000000D539000000000000D539000057
:10414C0000000000D539000000000000D539000047
:10415C0000000000D539000000000000D539000037
:10416C0000000000D539000000000000D539000027
:10417C0000000000D539000000000000D539000017
:10418C0000000000D539000000000000D539000007
:10419C0000000000D539000000000000D5390000F7
:1041AC0000000000D539000000000000D5390000E7
:1041BC0000000000D539000000000000D5390000D7
:1041CC0000000000D539000000000000D5390000C7
:1041DC0000000000D539000000000000D5390000B7
:1041EC0000000000D539000000000000D5390000A7
:1041FC0000000000D539000000000000D539000097
:10420C0000000000D539000000000000D539000086
:10421C0000000000D539000000000000D539000076
:10422C0000000000D539000000000000D539000066
:10423C0000000000D539000000000000D539000056
:10424C0000000000D539000000000000D539000046
:10425C0000000000D539000000000000D539000036
:10426C0000000000D539000000000000D539000026
:08427C0000000000D53900002C
:0C428400FFFFFFFFFFFFFFFFFFFFFFFF3A
:104290000338FDD870470000B10C000065390000FC
:1042A0008D390000000000008F380000290C00004C
:1042B0008D0C00005F3900005339000059390000AF
:1042C0004D390000DD0A0000950A000000000000E2
:1042D00000000000CF39000009100000C90F0000E5
:1042E00071100000A90F00001C0000200400002035
:1042F00014000020000000000C000020020000005C
:104300000443000000000000CB4400000600000051
:10431000E0FF0F0000000020D34400002100000057
:10432000E0FF0620D91800003B3B0000473B00009F
:10433000593B0000633B00006D3B0000C9190000C1
:104340007B3B000000000000FFFFFFFF00258450C2
:1043500000000000FFFF0000002884500100000062
:104360008B3C0000B13C00007D3C00005D1C000067
:104370006D3C00000080005006000000FC3F000083
:10438000344000003C4000005C4000005C40000005
:10439000F5FFFFFFFF8FFFFFFF8FFFFFFE8FFFFF88
:1043A000FE8FFFFFFD8FFFFFFC8FFFFFFC8FFFFFE6
:1043B000FB8FFFFF6D757465785F667265652063BE
:1043C000616C6C65642077697468204E554C4C2094
:1043D000706172616D6574657200000043616E27E3
:1043E0007420696E697469616C697A65206D757491
:1043F00065782C20776173204E554C4C0D0A0000D7
:10440000436F756C64206E6F74206C6F636B2070EB
:104410006F7765722073617665206D7574657800BD
:104420004750494F5F3000303132333435363738FA
:1044300039616263646566004661696C6564207415
:104440006F207265626F6F743A207370696E6E6967
:104450006E6720656E646C6573736C792E2E2E0A00
:1044600000554152545F3000434C4F434B00737929
:10447000735F636C6F636B006D757465785F696EF5
:1044800069742063616C6C65642077697468204E80
:10449000554C4C20706172616D6574657200436F9C
:1044A000756C64206E6F7420616C6C6F63617465F1
:1044B000206D75746578206265666F726520696E1F
:1044C000697469616C697A696E6700464C4153484A
:1044D0005F30005352414D5F30004750494F5F31CC
:1044E0000048575F43433358585F300076322E34CC
:1044F0002E302D6E637332002A2A2A20426F6F7489
:10450000696E67205A6570687972204F5320627512
:10451000696C64202573202573202A2A2A0A006DDD
:0445200061696E005F
:104524000D3500000C0100200100000020010020D6
:1045340001000000340100200100000048010020B7
:1045440001000000053B00000000000000C2010063
:104554000001030000000000000000000090D003F0
:10456400400000204000002000000000A1320000B4
:10457400B8080020010000002533000001330000CA
:1045840045330000E13200008C0000205000002080
:1045940084000020000000007C000020BC080020F3
:1045A40001000000C008002001000000C408002031
:1045B400010000006C000020780000207000002042
:0845C400680000209C000020AB
:1045CC0068440000AC420000984200007C020020CD
:1045DC006144000074430000604300002800002088
:1045EC006E4400000000000000000000000000000D
:1045FC002044000048430000244300003008002001
:10460C00DA44000054430000244300004C0800200E
:10461C00E144000000000000000000000000000069
:04462C00000000008A
:104630000C0100200C010020000000000000000020
:104640000F000000200100202001002000000000D9
:10465000000000000F0000003401002034010020A1
:1046600000000000000000000F00000048010020D2
:104670004801002000000000000000000F000000C2
:0400000300001319CD
:00000001FF
